:100000000C9410050C9457050C9457050C94570547
:100010000C9457050C9457050C9457050C945705F0
:100020000C9457050C9457050C94640C0C94360DE5
:100030000C94A11B0C9457050C9457050C94570570
:100040000C9457050C9457050C9457050C945705C0
:100050000C9457050C94411C0C9457050C945705AF
:100060000C9457050C9457050C9457050C945705A0
:100070000C9457050C9457050C9457050C94570590
:100080000C9457050C9457050C9457050C94570580
:100090000C9457050C9457050C9457050C94570570
:1000A0000C9457050C9457050C945705A30DC50DDA
:1000B000B30EC50DB30E0A0E2D0EB30E820E950EA5
:1000C000AA11AA11D811D811351273128C148C14DC
:1000D0008C128C148D138D1360148C148C14771463
:1000E0001F141A16041D1B062021150807091905DF
:1000F00022231C170A0B11801E352B39797A7B2C91
:100100002425180C0E0D1080742A31287C7D7E7FEA
:1001100026271213330F36802D2E302F3438378098
:100120004B6579626F6172642073746172742E0A18
:100130000055534220636F6E666967757265642E61
:100140000A000D0A696E69740A005B445D005B4336
:100150005D001203480048004B00420020006D0083
:100160006F00640000000E0374002E006D002E006E
:100170006B002E0000000403090409028D00050134
:1001800000A032090400000103010100092111014E
:1001900000012240000705810308000A090401004C
:1001A0000103010200092111010001224D00070590
:1001B000820308000A09040200010300000009216B
:1001C000110100012236000705830308000A090413
:1001D0000300020300000009211101000122220096
:1001E000070584032000010705040320000109041A
:1001F000040001030000000921110100012239005F
:10020000070585032000011201100100000008ED20
:10021000FEFECA04010102000105010906A1010553
:100220000719E029E71500250195087501810205E8
:10023000081901290595057501910295017503912C
:10024000010507190029F71500250195F8750181A9
:1002500002C00631FF0974A1010975150026FF00CF
:100260009520750881020976150026FF00952075F6
:10027000089102C005010980A101850216810026AE
:10028000B7001A81002AB700751095018100C005DA
:100290000C0901A1018503160100269C021A010028
:1002A0002A9C02751095018100C005010902A10177
:1002B0000901A10005091901290515002501950568
:1002C000750181029501750381010501093009312C
:1002D0001581257F95027508810609381581257FCE
:1002E000950175088106050C0A38021581257F9550
:1002F0000175088106C0C005010906A1010507199D
:10030000E029E71500250195087501810295017521
:1003100008810105081901290595057501910295C6
:1003200001750391010507190029FF150026FF003B
:10033000950675088100C0636F6E73756D65723ABE
:1003400020253034580A0073797374656D3A20257E
:100350003034580A000A002530325820006B657985
:10036000626F6172643A20004C45443A2025303275
:10037000580A00253032583A202530386225730A51
:1003800000722F632030313233343536370A00643F
:10039000656C5F6B65795F6269743A2063616E2793
:1003A000742064656C3A20253032580A0061646418
:1003B0005F6B65795F6269743A2063616E277420B0
:1003C0006164643A20253032580A004F6E657368C4
:1003D0006F743A2074696D656F75740A00290A009C
:1003E0002575002F002575005D280025640020007C
:1003F000256400200025640020002564007C002581
:10040000303258006D6F7573656B6579205B62746F
:100410006E7C782079207620685D287265702F6167
:10042000636C293A205B006D6B5F776865656C5F74
:1004300074696D655F746F5F6D6178203D20256420
:100440000A006D6B5F776865656C5F6D61785F73DF
:1004500070656564203D2025640A006D6B5F7469DA
:100460006D655F746F5F6D6178203D2025640A00C3
:100470006D6B5F6D61785F7370656564203D2025ED
:10048000640A006D6B5F696E74657276616C203D05
:100490002025640A006D6B5F64656C6179203D20E6
:1004A00025640A006D6B5F776865656C5F74696DC4
:1004B000655F746F5F6D6178203D2025640A006D73
:1004C0006B5F776865656C5F6D61785F737065659C
:1004D00064203D2025640A006D6B5F74696D655F63
:1004E000746F5F6D6178203D2025640A006D6B5F3D
:1004F0006D61785F7370656564203D2025640A0036
:100500006D6B5F696E74657276616C203D20256449
:100510000A006D6B5F64656C6179203D2025640A7B
:10052000000A00257500363A20776865656C5F74AF
:10053000696D655F746F5F6D61783A20000A002510
:100540007500353A20776865656C5F6D61785F731B
:10055000706565643A20000A00257500343A2074FD
:10056000696D655F746F5F6D61783A20000A0025E0
:100570007500333A206D61785F73706565643A2069
:10058000000A00257500323A20696E746572766142
:100590006C286D73293A20000A00257500313A2035
:1005A00064656C6179282A31306D73293A20000A1C
:1005B000092D2056616C756573202D0A004D3E0093
:1005C0004D25643E20003F007365742064656661BC
:1005D000756C740A00433E2000776865726520647C
:1005E000656C74613A20637572736F723D25642C7B
:1005F00020776865656C3D25640A536565206874DD
:1006000074703A2F2F656E2E77696B697065646917
:10061000612E6F72672F77696B692F4D6F757365E8
:100620005F6B6579730A000A092D204D6F7573653C
:100630006B6579202D0A4553432F713A097175690D
:10064000740A313A0964656C6179282A31306D7316
:10065000290A323A09696E74657276616C286D7385
:10066000290A333A096D61785F73706565640A34ED
:100670003A0974696D655F746F5F6D61780A353A28
:1006800009776865656C5F6D61785F737065656437
:100690000A363A09776865656C5F74696D655F74E1
:1006A0006F5F6D61780A0A703A097072696E742022
:1006B00076616C7565730A643A09736574206465C4
:1006C0006661756C74730A75703A092B310A646F30
:1006D000776E3A092D310A706775703A092B3130FF
:1006E0000A7067646F776E3A092D31300A0A7370A9
:1006F000656564203D2064656C7461202A206D610D
:10070000785F7370656564202A2028726570656162
:1007100074202F2074696D655F746F5F6D61782937
:100720000A003F004D3E2000433E20004C25640A55
:10073000000A092D20436F6E736F6C65202D0A45EA
:1007400053432F713A09717569740A6D3A096D6FD7
:100750007573656B65790A000A092D204D6167691B
:1007600063202D0A643A0964656275670A783A095C
:100770006465627567206D61747269780A6B3A0905
:100780006465627567206B6579626F6172640A6D7A
:100790003A096465627567206D6F7573650A763A0C
:1007A0000976657273696F6E0A733A0973746174BE
:1007B00075730A633A09636F6E736F6C65206D6FB2
:1007C00064650A302D343A096C61796572302D34D4
:1007D000284631302D4634290A506175733A096232
:1007E0006F6F746C6F616465720A6E3A094E4B529A
:1007F0004F0A003F004E4B524F3A206F66660A0088
:100800004E4B524F3A206F6E0A0074696D65725FED
:1008100072656164333228293A202530346C580AD5
:10082000006B6579626F6172645F6E6B726F3A2004
:1008300025580A006B6579626F6172645F69646C48
:10084000653A2025580A006B6579626F6172645FB2
:1008500070726F746F636F6C3A2025580A00686F6E
:1008600073745F6B6579626F6172645F6C656473EA
:1008700028293A2025580A000A092D20537461744A
:100880007573202D0A004743433A20342E392E3207
:10089000204156522D4C4942433A20312E382E30B9
:1008A00073766E204156525F415243483A2061763A
:1008B00072350A004F5054494F4E533A204C55461A
:1008C00041204D4F5553454B4559204558545241B1
:1008D0004B455920434F4E534F4C4520434F4D4DB0
:1008E000414E44204E4B524F204B45594D41505F95
:1008F00053454354494F4E20343039360A0042554F
:10090000494C443A20353732633236352D646972AA
:100910007479202831343A33303A3534204A616EC4
:100920002032352032303137290A005649443A20E6
:1009300030784645454428742E6D2E6B2E29205064
:1009400049443A203078434146452848484B4220A4
:100950006D6F6429205645523A203078303130345A
:100960000A00444553433A20742E6D2E6B2E206BA3
:100970006579626F617264206669726D7761726514
:1009800020666F722048484B42206D6F640A000A4F
:10099000092D2056657273696F6E202D0A000A6D4D
:1009A0006F7573653A206F66660A000A6D6F75731E
:1009B000653A206F6E0A000A6B6579626F61726436
:1009C0003A206F66660A000A6B6579626F6172642D
:1009D0003A206F6E0A000A6D61747269783A206F6E
:1009E00066660A000A6D61747269783A206F6E0A51
:1009F000000A64656275673A206F6E0A000A6465D2
:100A00006275673A206F66660A000A0A626F6F7441
:100A10006C6F616465722E2E2E2000433E20000014
:100A200011241FBECFEFDAE0DEBFCDBF04B603FE58
:100A300027C080910A0290910B02A0910C02B09104
:100A40000D028730904BA740B04BD1F410920A02B0
:100A500010920B0210920C0210920D0214BE84B779
:100A6000877F84BF0FB6F894A89580916000886155
:100A700080936000109260000FBEE0E0F8E30995FB
:100A800011E0A0E0B1E0E8E9F9E402C005900D92C0
:100A9000A833B107D9F722E0A8E3B1E001C01D9265
:100AA000AA30B207E1F70E9492090C94CA240C9470
:100AB0000000FF93EF93E0913801F09139013097F6
:100AC00009F00995EF91FF910895FC01859180301F
:100AD00011F0EFDFFBCF0895FF27E0E230E247FFA0
:100AE0000CC0419597FF09C0EDE260957095809527
:100AF0009095611D711D811D911D27FF02C02195DB
:100B000030E350E2AA27660F771F881F991FAA1F9C
:100B1000A41710F0A41B63955A95A9F7AA3008F002
:100B2000A95FA05DAF93F3956115710581059105EE
:100B300041F7ED3211F4EF93F395F21718F43F9368
:100B4000F395FBCF8F91B5DFFA95E1F70895E99121
:100B5000F9918591803021F0853219F0AADFF9CF23
:100B6000089520E0E89455915532C1F3503311F4C3
:100B7000689455915A3348F4505390F3220F022E43
:100B8000220F220F200D250FF4CF0EF4219589910D
:100B90009991533619F3533729F1533559F1BC0163
:100BA00088279927E8945C3621F489919991689473
:100BB0005591543639F446EF7EF077FF0DC08FEF34
:100BC0009FEF0AC055374AE039F0583540E121F02F
:100BD000523642E009F00895FF93EF937DDFEF91E5
:100BE000FF91B7CFFF93EF93FC0181918030B9F370
:100BF00060DFFBCFFF93EF9368DFF1CFDF93CF93FD
:100C0000CDB7DEB72596A3DFCF91DF9108958FEFA3
:100C100084B980E485B957985F9A87B18F7387B993
:100C200088B1806C88B92E9A2F98E2E4F1E088E0D0
:100C30008E0F11928E13FDCFEAE3F1E088E08E0F64
:100C400011928E13FDCF82E491E090934D01809339
:100C50004C018AE391E090934B0180934A010895FF
:100C60000F931F93CF93DF9380914A0190914B0193
:100C700020914C0130914D0130934B0120934A015A
:100C800090934D0180934C01C0E0D0E001E010E072
:100C900080E090E025B1207C2C2BAC0133E0440FA8
:100CA000551F3A95E1F7242B25B9EAE1EA95F1F7CA
:100CB00000C0E0914A01F0914B01EC0FFD1F208133
:100CC00030E0082E02C0359527950A94E2F720FD02
:100CD0002F9AF5E3FA95F1F70000E6B52E982AE190
:100CE0002A95F1F700C040914C0150914D01DA0175
:100CF000AC0FBD1F4F9B0AC09801082E01C0220FE8
:100D00000A94EAF720953C91232308C06C9198013E
:100D1000082E01C0220F0A94EAF7262B2C9326B541
:100D20006E2F70E02E1718F026B530E004C026B5FF
:100D300030E021503F4F261B370B2630310558F04D
:100D4000E0914A01F0914B01EC0FFD1F2081FA0167
:100D5000EC0FFD1F20833AE13A95F1F700C02F9880
:100D60002E9AEBE2F1E03197F1F700C00000019616
:100D70008830910509F08ECFA0914C01B0914D01C2
:100D8000AC0FBD1FE0914A01F0914B01EC0FFD1F2C
:100D90009C918081981751F00E94DF1B60934E0157
:100DA00070934F0180935001909351012196C83068
:100DB000D10509F06DCF80910102853021F080913D
:100DC0000102811111C060914E0170914F0180911B
:100DD0005001909151010E94151C613177428105AB
:100DE000910510F00E94601B81E0DF91CF911F916F
:100DF0000F91089520914C0130914D01F901E80FB8
:100E0000F11D8081089508950895569A81FF02C0CA
:100E10005E9A08955E9808958091760108959FB72F
:100E2000F894109255019FBF90910102943009F0FF
:100E300057C09091E9009F703091EC00232F2170F2
:100E400030FD20E8922B24E02093E9002091EB0074
:100E500020FF43C02091EE0027FF3FC020915201A8
:100E6000222321F02091E80025FF37C01092520183
:100E700026E03091E80035FD15C030910102343094
:100E800061F53091EB0035FD28C0215021F481E05F
:100E90008093520122C0EFE9FFE03197F1F700C0E3
:100EA0000000E7CF8093F1008091E80085FD0AC043
:100EB0008091E80080FFFCCF8091E8008E778093DE
:100EC000E80006C08FB7F89421E0209355018FBF4A
:100ED0009F709093E90080E008959F709093E900DF
:100EE0008FEF0895CF93DF9300D01F92CDB7DEB779
:100EF0009C0180910102843019F593E099833B8332
:100F00002A839093E9008FEF9091E800815095FD3E
:100F100006C095ED9A95F1F700008111F5CF80910B
:100F2000E80085FF0DC040E050E063E070E0CE01D6
:100F300001960E94540A8091E8008E778093E80021
:100F40000F900F900F90DF91CF910895CF93DF9383
:100F500000D01F92CDB7DEB720910102243021F5D9
:100F600022E029839B838A8383E08093E9008FEFCB
:100F70009091E800815095FD06C095ED9A95F1F7A6
:100F800000008111F5CF8091E80085FF0DC040E0A1
:100F900050E063E070E0CE0101960E94540A809117
:100FA000E8008E778093E8000F900F900F90DF910C
:100FB000CF910895209101022430F1F422E0209392
:100FC000E9002FEF3091E800215035FD06C035EDE6
:100FD0003A95F1F700002111F5CF2091E80025FFA7
:100FE0000BC040E050E065E070E00E94540A809140
:100FF000E8008E778093E8000895CF93DF932091E7
:101000000102243009F048C0EC0180910A018823D4
:10101000E1F080910B018823C1F085E08093E90025
:101020008FEF9091E800815095FD06C095E19A956B
:10103000F1F700008111F5CF8091E80085FF2CC009
:1010400040E050E060E270E017C081E08093E9008A
:101050008FEF9091E800815095FD06C095ED9A952F
:10106000F1F700008111F5CF8091E80085FF14C0F1
:1010700040E050E068E070E0CE010E94540A8091A8
:10108000E8008E778093E80080E2FE01A6E5B1E0FB
:1010900001900D928A95E1F7DF91CF9108958EE44A
:1010A00091E00E94650580910002811109C00E94B3
:1010B000E90B0E94460C8091E20084608093E2007C
:1010C00008958AE491E00E94650510920002089557
:1010D0000895209153012F5F822F62E30E94902494
:1010E000992319F020935301089510925301809190
:1010F0005501882371F180910102843041F580917E
:10110000E9008F702091EC00922F917020FD90E803
:10111000892B94E09093E9009091EB0090FF14C02C
:101120009091EE0097FF10C09091E80095FF03C0EA
:101130001092F100F9CF9091E80090FF05C09091D6
:10114000E8009E779093E8008F708093E9001092FA
:101150005501089542E061EC81E00E94630B42E09A
:1011600061EC82E00E94630B42E061EC83E00E944C
:10117000630B42E261EC84E00E94630B42E261ECAB
:1011800085E00C94630B80910302833009F455C011
:1011900030F4813071F0823009F48EC008958A30C5
:1011A00009F47AC08B3009F460C0893009F09CC022
:1011B00020C080910202813A09F096C08091E80037
:1011C000877F8093E8008091060290910702892B27
:1011D00021F460E286E591E003C060E080E090E009
:1011E00070E00E949F0A8091E8008B778093E8006E
:1011F000089580910202813209F076C08091060242
:1012000090910702009719F0049709F06DC0809142
:10121000E800877F8093E8008091E80082FD05C0A8
:10122000809101028111F8CF5FC08091F10080931D
:1012300076018091E8008B7753C080910202813A59
:1012400009F052C08091060290910702892B09F0A3
:101250004BC08091E800877F8093E8008091E80090
:1012600080FFFCCF80910A0136C08091020281325A
:10127000D9F58091060290910702892BA9F58091FA
:10128000E800877F8093E8000E94980B8091040219
:1012900080930A010C94AE1480910202813221F5F0
:1012A0008091E800877F8093E8000E94980B8091EE
:1012B000050280937701089580910202813AA1F49A
:1012C0008091E800877F8093E8008091E80080FFAC
:1012D000FCCF809177018093F1008091E8008E77B8
:1012E0008093E8000C94980B0895089508958091D8
:1012F0007601809354011092760180E00E940507E8
:101300000E9451100C94AE140C9477090E94601B3B
:101310008091FF01882329F00E94891B81110C9480
:101320003E0A089584B7877F84BF0FB6F894A895C6
:1013300080916000886180936000109260000FBE11
:1013400090E080E80FB6F89480936100909361007C
:101350000FBE8FE097E00E94311B82E491E00E9473
:1013600065050E9475090E948C0F0E94E90B0E947E
:10137000460C8091E20084608093E2007894809132
:1013800001028430E1F781E391E00E9465050E944B
:101390008E0F80E091E00E94CB0E80E291E00E94EF
:1013A00065050E94760980910102853019F40E943A
:1013B0008609F9CF0E94920FF6CF0E949D1B809163
:1013C00054018093760108950C94DD09292F332769
:1013D00023303105C9F064F42130310581F0223029
:1013E000310509F043C08DE890E02AE731E042C0C2
:1013F00021323105F1F02232310541F137C082E16D
:1014000090E027E032E036C099278130910541F025
:101410008230910541F0892B49F5E6E7F1E005C0FE
:10142000E6E6F1E002C0E2E5F1E0849190E09F01A0
:1014300021C06530D8F4E62FF0E0EE0FFF1FED5D20
:10144000FE4F2081318189E090E014C0653070F456
:1014500070E0FB01EE0FFF1FE75EFE4F2081318140
:10146000FB01EC5EFE4F808190E004C080E090E0E4
:1014700020E030E0FA0131832083089580E189BDC6
:1014800082E189BD09B400FEFDCF8091D8008F7D37
:101490008093D8008091E00082608093E00080918A
:1014A000E00081FDFCCF0895CF92DF92EF92FF9292
:1014B0000F931F93CF93DF93EC018B016A010E947E
:1014C000B70B811133C0C114D10439F0F60180810A
:1014D0009181081B190BC80FD91FE12CF12C0115A4
:1014E000110519F18091E80085FD16C08091E80092
:1014F0008E778093E800C114D10449F0F601808111
:101500009181E80EF91EF182E08285E00FC00E9411
:10151000B70B882321F30AC089918093F100015011
:101520001109FFEFEF1AFF0ADACF80E0DF91CF91C8
:101530001F910F91FF90EF90DF90CF900895209131
:101540000802309109022617370748F06115710526
:1015500039F42091E8002E772093E80001C0B9010A
:1015600040E061157105A9F120910102222309F4DF
:1015700043C0253009F442C02091E80023FD40C05B
:101580002091E80022FD32C02091E80020FFE9CF41
:101590004091F3002091F20030E0342BFC01CF01A8
:1015A0006115710559F02830310540F4819180931F
:1015B000F100615071092F5F3F4FF1CF41E02830BA
:1015C000310509F040E02091E8002E772093E800F3
:1015D000C8CF4111C9CF0AC080910102882361F0B0
:1015E000853061F08091E80083FD0AC08091E800B9
:1015F00082FFF2CF80E0089582E0089583E00895AD
:1016000081E00895209108023091090226173707DA
:1016100048F06115710539F42091E8002E77209388
:10162000E80001C0B901FC0120E06115710591F1EC
:1016300080910102882309F440C0853009F43FC03D
:101640008091E80083FD3DC08091E80082FD2FC0BD
:101650008091E80080FFE9CF2091F3008091F200B3
:1016600090E0922B6115710559F08830910540F496
:1016700024912093F1003196615071090196F2CFC7
:1016800021E0089709F020E08091E8008E778093B0
:10169000E800CBCF2111CCCF0AC080910102882372
:1016A00061F0853061F08091E80083FD0AC080918F
:1016B000E80082FFF2CF80E0089582E0089583E0A1
:1016C000089581E00895982F973058F59093E90098
:1016D000981739F07091EC002091ED005091F000D6
:1016E00003C0242F762F50E021FF19C03091EB006A
:1016F0003E7F3093EB003091ED003D7F3093ED0065
:101700003091EB0031603093EB007093EC0020934C
:10171000ED005093F0002091EE0027FF07C09F5F7F
:10172000D3CF8F708093E90081E0089580E0089521
:101730008091020287FF11C08091E80082FD05C000
:10174000809101028111F8CF11C08091E8008B7760
:101750000BC080910102882349F08091E80080FF4E
:10176000F8CF8091E8008E778093E800089520916B
:10177000E4003091E50095E64091EC00842F817003
:1017800040FF22C08091E80080FD1CC080910102D2
:10179000882391F0853091F08091EB0085FD10C099
:1017A0004091E4005091E5004217530729F39A0154
:1017B000915011F784E0089582E0089583E0089540
:1017C00081E0089580E008954091E80042FFDECF77
:1017D00008950E94570C0E945F0CE0EEF0E08081BB
:1017E00081608083E8EDF0E080818F77808319BC91
:1017F000A7EDB0E08C918E7F8C9380818F7E80836B
:101800001092000208950F931F93CF93DF930E94CD
:10181000570C0E945F0CC8EDD0E088818F778883D9
:1018200088818068888388818F7D888319BC109225
:1018300001021092FD011092FF011092FE0100EED4
:1018400010E0F80180818B7F8083888181608883AC
:1018500042E060E080E00E94630BE1EEF0E0808116
:101860008E7F8083E2EEF0E08081816080838081E2
:1018700088608083F80180818E7F80838881806189
:101880008883DF91CF911F910F910895E8EDF0E0EB
:1018900080818F7E8083E7EDF0E0808181608083AE
:1018A00084E082BF81E0809300020C94030CE8ED99
:1018B000F0E080818E7F80831092E2000895109284
:1018C000DA001092E10008951F920F920FB60F9266
:1018D00011242F933F934F935F936F937F938F9335
:1018E0009F93AF93BF93EF93FF938091E10082FFAB
:1018F0000BC08091E20082FF07C08091E1008B7FE6
:101900008093E1000E9469088091DA0080FF1FC087
:101910008091D80080FF1BC08091DA008E7F809379
:10192000DA008091D90080FF0DC080E189BD82E19D
:1019300089BD09B400FEFDCF81E0809301020E94C1
:101940004F0805C019BC109201020E9461088091E5
:10195000E10080FF19C08091E20080FF15C08091F6
:10196000E2008E7F8093E2008091E20080618093AC
:10197000E2008091D80080628093D80019BC85E095
:10198000809301020E9484098091E10084FF30C0AD
:101990008091E20084FF2CC080E189BD82E189BD95
:1019A00009B400FEFDCF8091D8008F7D8093D800D0
:1019B0008091E1008F7E8093E1008091E2008F7E34
:1019C0008093E2008091E20081608093E200809148
:1019D000FD01882311F084E007C08091E30087FDBA
:1019E00002C081E001C083E0809301020E94E4090B
:1019F0008091E10083FF29C08091E20083FF25C030
:101A00008091E100877F8093E10082E08093010272
:101A10001092FD018091E1008E7F8093E100809122
:101A2000E2008E7F8093E2008091E20080618093EB
:101A3000E20042E060E080E00E94630B8091F000F1
:101A400088608093F0000E946808FF91EF91BF9139
:101A5000AF919F918F917F916F915F914F913F9146
:101A60002F910F900FBE0F901F9018951F920F92FD
:101A70000FB60F9211242F933F934F935F936F9361
:101A80007F938F939F93AF93BF93CF93DF93EF9306
:101A9000FF93C091E900CF708091EC00D82FD170F6
:101AA00080FDD0E81092E9008091F000877F80935C
:101AB000F00078940E947A0D1092E9008091F00075
:101AC00088608093F000CD2BCF70C093E900FF9128
:101AD000EF91DF91CF91BF91AF919F918F917F91C6
:101AE0006F915F914F913F912F910F900FBE0F908B
:101AF0001F9018951F93CF93DF93CDB7DEB7AA97AA
:101B00000FB6F894DEBF0FBECDBFE2E0F2E088E092
:101B10008E0F9091F10091938E13FBCF0E94C3081A
:101B20008091E80083FF1FC180910202909103021F
:101B3000492F50E04A30510508F015C1FA01EA5A20
:101B4000FF4F0C94B024803881F0823809F00BC12B
:101B5000809106028F708093E9008091EB0085FBF5
:101B6000882780F91092E90006C08091FE019091CB
:101B7000FF01911182609091E800977F9093E800B7
:101B80008093F1001092F100C8C0282F2D7F09F03A
:101B9000EAC0882319F0823061F0E5C08091040228
:101BA000813009F0E0C0933009F080E08093FF01BC
:101BB0002BC080910402811127C0809106028F7092
:101BC00009F4D1C08093E9002091EB0020FF1CC0F4
:101BD000933021F48091EB00806214C09091EB006F
:101BE00090619093EB0021E030E0A90102C0440F26
:101BF000551F8A95E2F74093EA001092EA0080911F
:101C0000EB0088608093EB001092E9008091E8007F
:101C1000877F86C08111A7C0109104021F77809131
:101C2000E3008078812B8093E3008091E800877F38
:101C30008093E8000E94980B8091E80080FFFCCF21
:101C40008091E30080688093E300111102C082E07C
:101C500001C083E08093010286C08058823008F082
:101C600082C080910402909105028C3D53E095075B
:101C700079F583E08A838AE289834FB7F894DE019D
:101C8000139620E03EE051E2E32FF0E0509357003E
:101C9000E49120FF03C0E295EF703F5FEF708E2F5D
:101CA00090E0EA3010F0C79601C0C0968D939D93E6
:101CB0002F5F243149F74FBF8091E800877F8093E1
:101CC000E8006AE270E0CE0101960E949F0A14C00B
:101CD000AE014F5F5F4F609106020E94E609BC01B2
:101CE000892B09F440C09091E800977F9093E80019
:101CF00089819A810E94020B8091E8008B77809302
:101D0000E80031C0803879F58091E800877F8093C2
:101D1000E8008091FD018093F1008091E8008E77CA
:101D20008093E8000E94980B1EC081111CC0909106
:101D300004029230C0F48091E800877F8093E8002D
:101D40009093FD010E94980B8091FD01811106C0C6
:101D50008091E30087FD02C081E001C084E08093B0
:101D600001020E94AA088091E80083FF0AC08091C6
:101D7000E800877F8093E8008091EB008062809389
:101D8000EB00AA960FB6F894DEBF0FBECDBFDF9171
:101D9000CF911F91089590937D0180937C010895C8
:101DA000E0917C01F0917D01309721F00190F0816C
:101DB000E02D099480E00895EF92FF920F931F9316
:101DC000CF93DF93E0917C01F0917D013097B1F1E9
:101DD0008C010280F381E02D09958091EC0182FF56
:101DE0002DC080FF04C08DE593E00E946505E801E9
:101DF00010E287E5E82E83E0F82E8091EC0180FF69
:101E00000BC088811F928F93FF92EF920E94FE0574
:101E10000F900F900F900F90115021961111EDCF50
:101E20008091EC0180FF0AC085E593E0DF91CF91BE
:101E30001F910F91FF90EF900C946505DF91CF916A
:101E40001F910F91FF90EF900895E0917C01F09128
:101E50007D01309721F00480F581E02D09940895EB
:101E6000CF93DF93EC0180917A0190917B01C817A9
:101E7000D90709F1D0937B01C0937A01E0917C01ED
:101E8000F0917D013097B9F00680F781E02DCE0109
:101E900009958091EC0182FF0EC080FF0CC0DF939A
:101EA000CF9387E493E09F938F930E94FE050F905A
:101EB0000F900F900F90DF91CF910895CF93DF9304
:101EC000EC018091780190917901C817D90709F147
:101ED000D0937901C0937801E0917C01F0917D016C
:101EE0003097B9F00084F185E02DCE0109958091FD
:101EF000EC0182FF0EC080FF0CC0DF93CF9387E31D
:101F000093E09F938F930E94FE050F900F900F9088
:101F10000F90DF91CF9108950C9452100E94CA1B2C
:101F20000C940706CF92DF92EF92FF920F931F93CC
:101F3000CF93DF9300D000D000D0CDB7DEB70E94A2
:101F400030068FE7C82E81E0D82E00E010E0E02EAA
:101F5000802F0E94FA06F60141916F01F42EF826B7
:101F6000B1F40F5F1F4F0830110589F78FEF898398
:101F70008A831B820E94D31B8160782F9D838C8370
:101F800049815A816B818D810E94871047C0909151
:101F9000EC0191FF04C08E830E9453108E8120E0DB
:101FA00030E04F2D50E0922FBA01022E02C07595FD
:101FB00067950A94E2F760FF2BC02983EA8221E04B
:101FC00030E0690102C0CC0CDD1C9A95E2F790E08C
:101FD0008C219D21892B09F420E02B830E94D31BA7
:101FE0008160782F9D838C8349815A816B818D819B
:101FF0000E94871049815A816B817C818D810E946A
:102000004D1BF801E158FE4F8081C826C08206C0F2
:102010002F5F3F4F2830310531F6A3CF0E944C1B74
:102020000E94C01E10917E010E94D00E181741F12F
:102030000E94D00E80937E019091EC0192FF0EC021
:1020400090FF0CC01F928F9388E693E09F938F932D
:102050000E94FE050F900F900F900F9080917E01CF
:1020600026960FB6F894DEBF0FBECDBFDF91CF919D
:102070001F910F91FF90EF90DF90CF900C945E1B1B
:1020800026960FB6F894DEBF0FBECDBFDF91CF917D
:102090001F910F91FF90EF90DF90CF9008950C94D7
:1020A000050708950895EF92FF920F931F93CF9322
:1020B000DF9381E893E00E946505C0E0D0E08DE207
:1020C000E82E81E0F82E03E713E08C2F0E94FA0639
:1020D0000E94361BFF92EF921F928F93DF93CF9354
:1020E0001F930F930E94FE0521968DB79EB7089609
:1020F0000FB6F8949EBF0FBE8DBFC830D10529F72B
:10210000DF91CF911F910F91FF90EF900895CF93A2
:10211000DF93CDB7DEB72B970FB6F894DEBF0FBEB7
:10212000CDBF942F4F83252F588769877A878B8758
:102130004A855B85452B21F02F3F09F59F3FF9F438
:10214000DE01119686E0FD0111928A95E9F785E09E
:10215000FE01379601900D928A95E1F749815A81E7
:102160006B817C818D819E810E9462172B960FB6B8
:10217000F894DEBF0FBECDBFDF91CF9108954F81A0
:10218000588569857A858B850E944D1BD9CFCF9361
:10219000882309F465C0C82F8CEF8C0F813A20F09A
:1021A00080E58C0F8E3248F48C2F0E940A22811118
:1021B00057C08C2F0E94ED190CC080E28C0F883024
:1021C00058F4C77081E001C0880FCA95EAF70E94F1
:1021D000981ACF910C94DC1A8BE58C0F833078F42D
:1021E000C53A29F0C63A31F083E890E005C081E8AD
:1021F00090E002C082E890E0CF910C94300F88E527
:102200008C0F853168F5C83A89F0C93A91F0CA3A1D
:1022100099F0CB3AA1F0CC3AA9F0CD3AB1F0CE3A50
:10222000B9F0CF3AC1F080E090E017C082EE90E0C4
:1022300014C089EE90E011C08AEE90E00EC085EBEC
:1022400090E00BC086EB90E008C083EB90E005C007
:1022500084EB90E002C087EB90E0CF910C945E0F8E
:10226000CF910895882349F19CEF980F913A20F07F
:1022700090E5980F9E3218F40E94401A0DC090E22B
:10228000980F983058F4877091E001C0990F8A95A3
:10229000EAF7892F0E949E1A0C94DC1A9BE5980F8E
:1022A000933020F480E090E00C94300F885A853110
:1022B00020F480E090E00C945E0F0895882321F0D4
:1022C0000E94981A0C94DC1A0895882321F00E9429
:1022D0009E1A0C94DC1A0895BF92CF92DF92EF926F
:1022E000FF920F931F93CF93DF9300D000D000D0C5
:1022F000CDB7DEB725E0FC01DE01119601900D920D
:102300002A95E1F7FC0140813181F28025812295F7
:102310002F7063817481672B09F4FEC23F3F19F46B
:102320004F3F09F4F9C26C0149833A8389819A814C
:102330002E830E94AC19182FB92E0E94AB190E944F
:10234000BB18EB2DE295EF70F0E0E05AFF4F2E81C5
:102350000C94B0248B2D807F9B2D9F70092F882398
:1023600011F00295007FFF2049F0002309F481C29B
:10237000802F0E94AB1A0E94DC1A7BC2812F0E9420
:102380003211002309F4C8C2802F0E94B11A269688
:102390000FB6F894DEBF0FBECDBFDF91CF911F9176
:1023A0000F91FF90EF90DF90CF90BF900C94DC1ACC
:1023B0008B2D807F9B2D9F70092F803211F002950D
:1023C000007F112319F0113009F12AC0FF20B1F06C
:1023D000802F222351F1213041F526960FB6F89433
:1023E000DEBF0FBECDBFDF91CF911F910F91FF9048
:1023F000EF90DF90CF90BF900C94BB1A222319F07E
:10240000213009F489C20E94C41A2DC0FF20F1F0C6
:10241000263008F081C20E94951A802329F023C03B
:10242000FF20F9F0211116C0802F26960FB6F894E0
:10243000DEBF0FBECDBFDF91CF911F910F91FF90F7
:10244000EF90DF90CF90BF900C945E11253008F094
:1024500063C209C0F601858180FF0BC28F7085833E
:10246000E3CF21111BC2802F82C12B2D26952695EB
:10247000237030E02115310521F021303105D1F0F4
:102480004BC2FF2021F0812F9B2D937002C080E072
:1024900090E026960FB6F894DEBF0FBECDBFDF9159
:1024A000CF911F910F91FF90EF90DF90CF90BF9051
:1024B0000C94300FFF2021F0812F9B2D937002C0D0
:1024C00080E090E026960FB6F894DEBF0FBECDBF39
:1024D000DF91CF911F910F91FF90EF90DF90CF9000
:1024E000BF900C945E0F812FFF2019F00E94461DB3
:1024F00002C00E94AE1D26960FB6F894DEBF0FBE36
:10250000CDBFDF91CF911F910F91FF90EF90DF90A2
:10251000CF90BF900C94331E8B2D837009F07BC03D
:10252000F110FAC1812F829586958770880F880FE8
:10253000912F9F70C92ED12CE12CF12C082E04C0B4
:10254000CC0CDD1CEE1CFF1C0A94D2F714FF12C049
:102550004FE050E060E070E004C0440F551F661F7C
:10256000771F8A95D2F7CB01BA0160957095809557
:10257000909503C060E070E0CB012B2D2695269549
:102580002370422F50E042305105D9F043305105BD
:1025900069F16C297D298E299F294130510551F11E
:1025A00026960FB6F894DEBF0FBECDBFDF91CF9158
:1025B0001F910F91FF90EF90DF90CF90BF900C9400
:1025C000D0186C297D298E299F2926960FB6F8945C
:1025D000DEBF0FBECDBFDF91CF911F910F91FF9056
:1025E000EF90DF90CF90BF900C94E2180E94D0182B
:1025F000C701B60126960FB6F894DEBF0FBECDBF59
:10260000DF91CF911F910F91FF90EF90DF90CF90CE
:10261000BF900C94BE18FF2019F08B2D817001C063
:102620008695882309F478C1812F829586958770D5
:10263000880F880F912F9F70C92ED12CE12CF12C7F
:10264000082E04C0CC0CDD1CEE1CFF1C0A94D2F733
:1026500014FF12C04FE050E060E070E004C0440F8F
:10266000551F661F771F8A95D2F7CB01BA01609577
:1026700070958095909503C060E070E0CB012B2DA4
:10268000269526952370422F50E042305105D9F00F
:102690004330510569F16C297D298E299F294130EC
:1026A000510551F126960FB6F894DEBF0FBECDBF8F
:1026B000DF91CF911F910F91FF90EF90DF90CF901E
:1026C000BF900C9487196C297D298E299F29269605
:1026D0000FB6F894DEBF0FBECDBFDF91CF911F9133
:1026E0000F91FF90EF90DF90CF90BF900C949919CD
:1026F0000E948719C701B60126960FB6F894DEBF6F
:102700000FBECDBFDF91CF911F910F91FF90EF9042
:10271000DF90CF90BF900C947519103FC9F128F449
:1027200080E4810F803250F09FC0123F09F461C0F5
:1027300008F44AC0133F09F471C096C0012F00711C
:102740008B2D8F71FF2051F00E940E19812F0023D5
:1027500019F08295807F69CE8F7067CE0E942F1905
:10276000812F002319F08295807F01C08F702696FB
:102770000FB6F894DEBF0FBECDBFDF91CF911F9192
:102780000F91FF90EF90DF90CF90BF900C94651168
:10279000FF20B1F0253008F0BFC08B2D8F71269639
:1027A0000FB6F894DEBF0FBECDBFDF91CF911F9162
:1027B0000F91FF90EF90DF90CF90BF900C94541941
:1027C000263008F0A9C0E9CFFF20A9F08B2D8F712A
:1027D00026960FB6F894DEBF0FBECDBFDF91CF9126
:1027E0001F910F91FF90EF90DF90CF90BF900C94CE
:1027F0000E19FF2059F38B2D8F7126960FB6F89482
:10280000DEBF0FBECDBFDF91CF911F910F91FF9023
:10281000EF90DF90CF90BF900C942F19FF2099F08C
:102820008B2D8F7126960FB6F894DEBF0FBECDBFED
:10283000DF91CF911F910F91FF90EF90DF90CF909C
:10284000BF900C94F91826960FB6F894DEBF0FBE11
:10285000CDBFDF91CF911F910F91FF90EF90DF904F
:10286000CF90BF900C94F418FF20A9F0222309F414
:10287000ADCF812F26960FB6F894DEBF0FBECDBF29
:10288000DF91CF911F910F91FF90EF90DF90CF904C
:10289000BF900C94C710222309F4ADCF812F269648
:1028A0000FB6F894DEBF0FBECDBFDF91CF911F9161
:1028B0000F91FF90EF90DF90CF90BF900C9432116A
:1028C0004B2D4F70612FC6010E94C01C26960FB67B
:1028D000F894DEBF0FBECDBFDF91CF911F910F9156
:1028E000FF90EF90DF90CF90BF900C9406184B2D87
:1028F0004F70612FC60126960FB6F894DEBF0FBE4B
:10290000CDBFDF91CF911F910F91FF90EF90DF909E
:10291000CF90BF900C94C31C26960FB6F894DEBFE0
:102920000FBECDBFDF91CF911F910F91FF90EF9020
:10293000DF90CF90BF9008950E94B81A0E94871A26
:102940000E94DC1A0E94651F0E94331E80E090E006
:102950000E94300F80E090E00C945E0F0E94A81A55
:102960000C949C140E94AC19292F22952F7030E0F2
:102970002C3031054CF42A303105C4F42250310991
:102980002230310540F023C02C303105D1F02F30FA
:102990003105B9F01CC0853A28F48430B0F4823097
:1029A00028F413C090E2980F983078F0883E30F405
:1029B000803E58F48450813A50F407C0803F39F487
:1029C00004C093FB882780F9089581E0089580E092
:1029D0000895CF93DF9300D000D01F92CDB7DEB71C
:1029E0000F900F900F900F900F90DF91CF9108955F
:1029F000CF93DF9300D000D000D0CDB7DEB72696BE
:102A00000FB6F894DEBF0FBECDBFDF91CF91089512
:102A10001F93CF93DF93C091870116E080918801C7
:102A2000C81799F0D0E01C9FF0011D9FF00D1124F4
:102A3000E757FE4F40815181628173818481958186
:102A40000E94F8142196C770E9CFDF91CF911F91B2
:102A500008954091B9015091BA016091BB01709104
:102A6000BC018091BD019091BE010C94F81480913D
:102A7000BE0182958F7009F054C08091BB018823FC
:102A800009F44FC080918701A09188016091B9013C
:102A90007091BA014091BC015091BD01B6E08A1716
:102AA00009F43FC090E041155105C1F17F3F11F499
:102AB0006F3FA1F1B89FF001B99FF00D1124E757C6
:102AC000FE4F218172132AC02081621327C0228108
:102AD000211124C0238134812417350710F421509B
:102AE0003109241B350B2C323140C0F42091BE013A
:102AF0002F7020612093BE0126E0289FF001299FBE
:102B0000F00D1124E257FE4F80818F708061808329
:102B100089EB91E00E946C110C9408150196877066
:102B2000BECF0895CF92DF92EF92FF920F931F9343
:102B3000CF93DF93CDB7DEB762970FB6F894DEBFC1
:102B40000FBECDBF8C0185E0F801DE011D9601901E
:102B50000D928A95E1F7D8014C9111965C911197ED
:102B600012966C9112971396CD90DC901497309139
:102B7000B9017091BA018091BC019091BD0100979B
:102B800009F473C17F3F19F43F3F09F46EC1E0902F
:102B9000BB01EE2009F4C5C02091BE01C816D906BC
:102BA00050F0F601E81BF90BCF01FF24F3948C32AF
:102BB0009140C8F009C0809590958C0D9D1DFF2413
:102BC000F3948C32914078F0F12C207F09F0C6C04C
:102BD0007C2DD98AC88A89890E94E91489EB91E001
:102BE0000E946C11B1C0822F807F09F045C075131F
:102BF00013C0341311C061110FC02F7020612093D6
:102C0000BE010E94291589EB91E00E946C11809110
:102C1000BE01F80185832EC0CD2819F15F3F11F464
:102C20004F3FF9F0F62E61111CC080918701209171
:102C3000880136E0821709F45BC090E0389FF0010C
:102C4000399FF00D1124E757FE4F7181571306C0CD
:102C50007081471303C07281711103C001968770A0
:102C6000E9CFF62E662309F41DC18091BE01816073
:102C70008093BE01F12C16C1751309C0341307C02F
:102C8000611105C08091BE01F8018583C8C04D87E0
:102C90005E878D859E856A8B0E94B2146A8988231F
:102CA000E1F16623D1F12091BE01822F82958F70D0
:102CB00090E0029774F08091B9019091BA019887E1
:102CC0008F831986DB86CA862C87CE0107960E94E1
:102CD0006C1186E0F801A9EBB1E001900D928A95A4
:102CE000E1F70E9437150E942915FF24F394DAC0FA
:102CF0004D875E878D859E850E94AC19292F229570
:102D00002F7030E0223031050CF0BFC09F7009F009
:102D1000B9C0805E883008F4C5C0C8010E946C113B
:102D2000E4CFC816D90608F453C0F601E81BF90B26
:102D3000CF018C32914008F453C0F12C7C2DD98AFC
:102D4000C88A89890E94E914E9EBF1E086E0DF0195
:102D50001D928A95E9F70E942915A4C0751314C025
:102D6000341312C0611110C08091BE01F801858337
:102D7000C8010E946C1186E0E9EBF1E0DF011D92D1
:102D80008A95E9F7FE2C8EC04D875E878D859E85DE
:102D90006A8B0E94B2146A89882309F4BECF662325
:102DA00009F4BBCF2091BE01822F82958F7090E0F5
:102DB00002970CF48ECF8091B9019091BA019A8359
:102DC00089831B82DD82CC822E83CE0101967FCF48
:102DD000809590958C0D9D1D8C32914008F0ADCF63
:102DE000F62E662309F499CF75132EC034132CC028
:102DF0002091BE0120FD1FC0822F82958F70D9F0D7
:102E0000D80115962C9315978F3049F08F5F982F26
:102E10009295907F822F8F70892B15968C93C80185
:102E20000E946C1186E0F801A9EBB1E001900D92CF
:102E30008A95E1F790CF86E0F801A9EBB1E0019027
:102E40000D928A95E1F72EC04D875E878D859E8510
:102E50000E94B21481113DCF8091BE0181608093A8
:102E6000BE01C8010E946C111DC0662309F455CF34
:102E70004D875E878D859E850E94B214882309F454
:102E80004CCF27CF811145CF0DC0243031050CF038
:102E900044CF9F7009F43DCFD80115969C91907F47
:102EA00009F037CF8F2D62960FB6F894DEBF0FBEB4
:102EB000CDBFDF91CF911F910F91FF90EF90DF90E9
:102EC000CF9008951F93CF93DF93CDB7DEB72C97A4
:102ED0000FB6F894DEBF0FBECDBF4F83588769870A
:102EE0007A878B879C87CE0107960E94921588234C
:102EF00069F08F8198852A853B85232BF1F19F3FCF
:102F000009F063C08F3F09F060C037C086E0FE0162
:102F10003796DE01119601900D928A95E1F76F8147
:102F20007885EA85FB85309741F17F3F11F46F3F4B
:102F300021F12091880130E0C9010196877099271D
:102F40004091870150E08417950709F447C06983D1
:102F50007A83FD83EC8396E0929FD001939FB00D1E
:102F60001124A757BE4FFE01319601900D929A95FC
:102F7000E1F7809388010E94081516E0809187018F
:102F8000909188018917C1F1189FC00111248757BA
:102F90009E4F0E949215882379F1E09187011E9F30
:102FA000F0011124E757FE4F408151816281738106
:102FB000848195810E94F8148091870190E00196A8
:102FC0008770992780938701D9CF4F81588569856C
:102FD0007A858B859C850E94F814CFCF0E94AE1411
:102FE0001092880110928701E9EBF1E086E0DF01A1
:102FF0001D928A95E9F7C1CF2C960FB6F894DEBFE3
:103000000FBECDBFDF91CF911F910895DF92EF9258
:10301000FF920F931F93CF93DF93FC01892B09F449
:103020008AC0E12CF12CDD24D394EF012196849108
:10303000853709F461C058F4843708F04EC08430F5
:1030400008F06AC08130D1F0823071F174C08837E5
:1030500009F45DC050F4863709F455C0873709F08C
:103060006AC08E2D0E94A51A54C09CE7980F903715
:1030700008F061C08F770E94321150C08F010E5F3F
:103080001F4FFE01849190E2980F983050F48770A2
:10309000FD2D01C0FF0F8A95EAF78F2F0E94AB1A12
:1030A00014C00E94C71013C08F010E5F1F4FFE0196
:1030B000C49180E28C0F883060F4C7708D2D01C000
:1030C000880FCA95EAF70E94B11A0E94DC1AE8013B
:1030D00025C08C2F0E943211FACF9F012E5F3F4FE7
:1030E000FE01C491CC2369F08FE99FE00197F1F7CD
:1030F00000C00000C150F6CF9F012E5F3F4FFE0180
:10310000F490E9010BC00E94951AE82E07C00E94B6
:10311000A81A0E94DC1A02C00E94C7108F2D8823B3
:1031200041F0EFE9FFE03197F1F700C00000815076
:10313000F6CFFE017ACFDF91CF911F910F91FF90D3
:10314000EF90DF9008956093C3017093C401809362
:10315000C5019093C6010E945C1B0C949C14609363
:10316000BF017093C0018093C1019093C2010E947E
:103170005D1B0C949C1408950C94A3180F931F933B
:103180000091C3011091C4012091C5013091C60185
:10319000602B712B822B932B1F910F910C94A318F2
:1031A0000F931F930091C3011091C4012091C50199
:1031B0003091C60160237123822393231F910F91C5
:1031C0000C94A3180F931F930091C3011091C40195
:1031D0002091C5013091C60160277127822793276E
:1031E0001F910F910C94A31860E070E0CB010C9438
:1031F000AF180F931F9341E050E060E070E08A0148
:103200009B0104C0000F111F221F331F8A95D2F7A4
:10321000C901B8011F910F910C94AF180F931F9320
:1032200041E050E060E070E004C0440F551F661FAD
:10323000771F8A95D2F78091BF019091C001A0912C
:10324000C101B091C2018A019B01082B192B2A2BC5
:103250003B2BC901B8011F910F910C94AF180F932C
:103260001F9341E050E060E070E004C0440F551F40
:10327000661F771F8A95D2F7409550956095709597
:103280008091BF019091C001A091C101B091C20194
:103290008A019B01082319232A233B23C901B80172
:1032A0001F910F910C94AF180F931F9341E050E0C2
:1032B00060E070E004C0440F551F661F771F8A95B9
:1032C000D2F78091BF019091C001A091C101B0914E
:1032D000C2018A019B01082719272A273B27C90118
:1032E000B8011F910F910C94AF180F931F93009189
:1032F000BF011091C0012091C1013091C201602B2A
:10330000712B822B932B1F910F910C94AF180F935D
:103310001F930091BF011091C0012091C101309114
:10332000C20160237123822393231F910F910C9478
:10333000AF180F931F930091BF011091C00120910E
:10334000C1013091C20160277127822793271F9105
:103350000F910C94AF180895CF92DF92EF92FF92E5
:103360000F931F93CF93DF938C01C090C301D09034
:10337000C401E090C501F090C6014091BF01509199
:10338000C0016091C1017091C201C42AD52AE62A08
:10339000F72ACFE1D0E0D701C6010C2E04C0B695C4
:1033A000A795979587950A94D2F780FF07C0B80133
:1033B0008C2F0E94961C8130910531F4219758F78B
:1033C000B80180E00E94961CDF91CF911F910F9170
:1033D000FF90EF90DF90CF90089590910A0199238C
:1033E00021F090910B01911109C020910C013091B5
:1033F0000D01F90132969FEF40E030C0982F96956D
:10340000969596959F31A0F4E0910C01F0910D01F5
:10341000E90FF11D877021E030E0A90102C0440FDF
:10342000551F8A95E2F7CA019181892B81830895FE
:103430009091EC0190FF23C01F928F938DEA93E04F
:103440009F938F930E94FE050F900F900F900F9007
:1034500008959F3F39F04F5F4E3141F0519158131D
:10346000F8CF0DC05111F7CF942FF5CF9F3F39F012
:10347000F901E90FF11D97FDFA95828308950895EA
:1034800090910A01992321F090910B01911109C0AB
:1034900020910C0130910D01F9013296205E3F4FD1
:1034A00030C0982F9695969596959F31A8F4E09107
:1034B0000C01F0910D01E90FF11D877021E030E062
:1034C000A90102C0440F551F8A95E2F7CA018095F1
:1034D00091818923818308959091EC0190FF16C01A
:1034E0001F928F938FE893E09F938F930E94FE0526
:1034F0000F900F900F900F9008953196E217F307F9
:1035000029F090819813F9CF1082F7CF089581E0C8
:1035100090E0E0910C01F0910D01E80FF91F10828D
:10352000019680329105A9F708958091EB010895E5
:103530009091EB01892B8093EB01089580959091F8
:10354000EB0189238093EB0108958093EB010895AB
:103550001092EB0108959091EA01892B8093EA0182
:10356000089580959091EA0189238093EA01089556
:103570001092EA0108958093C9010E94D31B909391
:10358000C8018093C70108951092C9011092C80123
:103590001092C701089580910C0190910D01FC01DA
:1035A00031969C01205E3F4F80E0919191118F5F99
:1035B000E217F307D1F70895E0910C01F0910D01A6
:1035C0008091EB018083E0910C01F0910D019081DD
:1035D0008091EA01892B80838091C9018823D9F1E8
:1035E0000E94D31B2091C7013091C8018217930715
:1035F00048F00E94D31B2091C7013091C801821B63
:10360000930B0AC00E94D31B2091C7013091C801BF
:1036100020953095820F931F8C32914070F08091ED
:10362000EC0180FF08C08BEC93E09F938F930E9486
:10363000FE050F900F900E94C41AE0910C01F091CA
:103640000D0190818091C901892B80830E94CB1A42
:1036500081110E94C41A80910C0190910D010C946B
:10366000DC0E909339018093380108958295982F4C
:103670009C7C392F36953695282F237344E0249F60
:10368000C0011124932F982B292F2A7A2695892F50
:103690008575880F822B08950895CF93DF9300D00E
:1036A00000D01F92CDB7DEB70F900F900F900F9004
:1036B0000F90DF91CF910895089508950C944F10C5
:1036C00080910102843021F11092ED0120E488E123
:1036D00090E00FB6F894A895809360000FBE2093F9
:1036E000600083B7817F846083BF83B7816083BFBD
:1036F0007894889583B78E7F83BF0FB6F894A8958A
:1037000080916000886180936000109260000FBE1D
:103710000895CF930E9403070E9430060E94040779
:10372000C0E08C2F0E94FA06811104C0CF5FC83020
:10373000C1F701C081E0CF9108950E9451100C940F
:10374000AE141F920F920FB60F9211248F939F9376
:10375000AF93BF938091ED01811113C08091EE0171
:103760009091EF01A091F001B091F1014196A11D5E
:10377000B11D8093EE019093EF01A093F001B093FF
:10378000F101BF91AF919F918F910F900FBE0F905C
:103790001F90189582E084BD93E095BD9AEF97BD88
:1037A00080936E0008952FB7F8948091EE01909168
:1037B000EF01A091F001B091F1012FBF08952FB753
:1037C000F8946091EE017091EF018091F001909179
:1037D000F1012FBF0895CF92DF92EF92FF920F93E6
:1037E0001F932FB7F8944091EE015091EF01609133
:1037F000F0017091F1012FBF6A017B01EE24FF24DB
:103800008C0120E030E0C016D106E206F30610F489
:10381000415051099A01281B390BC9011F910F9181
:10382000FF90EF90DF90CF900895CF92DF92EF92CC
:10383000FF920F931F932FB7F894C090EE01D09092
:10384000EF01E090F001F090F1012FBF97018601A8
:10385000061B170B280B390BC616D706E806F90608
:1038600018F0C901B80106C0C901B8016150710959
:10387000810991091F910F91FF90EF90DF90CF90F8
:1038800008951F920F920FB60F9211248F939F935A
:10389000AF93BF938091EE019091EF01A091F00161
:1038A000B091F1010196A11DB11D8093EE0190939D
:1038B000EF01A093F001B093F101BF91AF919F91FF
:1038C0008F910F900FBE0F901F9018950E94E90BDB
:1038D000F8942FEF87EA91E6215080409040E1F77D
:1038E00000C0000087E090EBDC0180930A02909317
:1038F0000B02A0930C02B0930D029CE088E10FB67E
:10390000F894A895809360000FBE90936000FFCF5D
:1039100028E0929FF0011124E80FF11DE052FF4FC3
:103920009491892F8F7092959F700895CF93C82F8F
:10393000CB010E94881C282F30E080E1989FA001D5
:103940001124422B532B4038510519F480E090E0AC
:1039500015C09770E92FF0E088E0C89FE00DF11DD9
:10396000112484E0EE0FFF1F8A95E1F7E20FF31FA9
:10397000EE0FFF1FE050F84985919491CF91089583
:1039800080E090E0089508958091F40180FF0BC0DD
:103990006091110185E0689FB001112475956795CC
:1039A000759567952BC081FF09C06091110185E075
:1039B000689FB00111247595679520C082FF07C0EC
:1039C0006091110185E0689FB001112417C09091AA
:1039D000F5019923D1F060911001961788F7209195
:1039E000110185E0289F90011124929FA001939FCF
:1039F000500D112470E0CA010E949C2460387105AA
:103A000040F46115710539F002C065E070E0862F61
:103A100008958FE7089581E008958091F40180FF73
:103A200008C060910F0170E0759567957595679571
:103A300021C081FF06C060910F0170E07595679508
:103A400019C082FF04C060910F0170E010C0909116
:103A5000F5019923C1F060910E019617A0F78091AE
:103A60000F01899FC001112470E00E949C246038DE
:103A7000710528F46115710521F0862F08958FE7EF
:103A8000089581E0089561E070E0F4CF803F21F473
:103A90000E94C41C819504C0813F29F40E94C41C6B
:103AA0008093F8010895823F21F40E94C41C8195FF
:103AB00004C0833F29F40E94C41C8093F701089539
:103AC000893F19F40E940D1D05C08A3F31F40E9400
:103AD0000D1D81958093F90108958B3F21F40E947B
:103AE0000D1D819504C08C3F29F40E940D1D80930B
:103AF000FA010895843F21F48091F601816017C096
:103B0000853F21F48091F601826011C0863F21F447
:103B10008091F60184600BC0873F21F48091F6010B
:103B2000886005C0883F31F48091F6018061809300
:103B3000F60108958D3F21F48091F40181600BC05E
:103B40008E3F21F48091F401826005C08F3F29F4FB
:103B50008091F40184608093F4010895803F39F4EA
:103B60008091F80187FF6CC01092F80169C0813F15
:103B700029F48091F8011816BCF362C09091F70106
:103B8000823F29F497FF5CC01092F70159C0833F30
:103B900019F41916CCF354C0893F41F48091F9010E
:103BA00018160CF04DC01092F9014AC08A3F29F452
:103BB0008091F90187FF44C0F6CF8B3F39F48091A3
:103BC000FA0187FF3DC01092FA013AC08C3F29F4F8
:103BD0008091FA011816BCF333C0843F21F4809120
:103BE000F6018E7F17C0853F21F48091F6018D7F0D
:103BF00011C0863F21F48091F6018B7F0BC0873F77
:103C000021F48091F601877F05C0883F31F48091CF
:103C1000F6018F7E8093F60113C08D3F21F48091D1
:103C2000F4018E7F0BC08E3F21F48091F4018D7FD3
:103C300005C08F3F29F48091F4018B7F8093F401BC
:103C40008091F70181110EC08091F80181110AC0A5
:103C50008091F901811106C08091FA01811102C0A1
:103C60001092F50108958091EC0183FF7EC084E0FD
:103C700094E00E9465058091F6011F928F938FEF6B
:103C800093E09F938F930E94FE058DEF93E00E9437
:103C900065058091F701282F082E000C330B3F9308
:103CA0008F938AEF93E09F938F930E94FE0588EF96
:103CB00093E00E9465058091F801282F082E000CE2
:103CC000330B3F938F9385EF93E09F938F930E94E5
:103CD000FE0583EF93E00E9465058091F901282F8E
:103CE000082E000C330B3F938F9380EF93E09F934C
:103CF0008F930E94FE058EEE93E00E9465058091F1
:103D0000FA01282F082E000C330B3F938F938BEE74
:103D100093E09F938F930E94FE0588EE93E00E94AC
:103D200065058091F5011F928F9385EE93E09F9337
:103D30008F930E94FE0583EE93E00E9465058091BB
:103D4000F4011F928F9380EE93E09F938F930E94D4
:103D5000FE058DED93E00E9465058DB79EB74C96EC
:103D60000FB6F8949EBF0FBE8DBF86EF91E00E9404
:103D7000250F0E94D31B9093F3018093F2010895C5
:103D80001F93CF93DF938091F2019091F3010E94F2
:103D9000EB1BAC019091F501992321F020911201C8
:103DA00030E006C0209113018AE0289F9001112481
:103DB0004217530708F485C08091F701C091F801BC
:103DC000D091F9011091FA01811107C0C11175C09C
:103DD000D11173C0111171C074C09F3F19F09F5F62
:103DE0009093F501181624F40E94C41C8093F701E7
:103DF0008091F70187FF05C00E94C41C81958093C4
:103E0000F7011C1624F40E94C41C8093F8018091D1
:103E1000F80187FF05C00E94C41C81958093F801BA
:103E20006091F701662331F1C091F801CC2311F1C3
:103E3000062E000C770B880B990B0E94972323E327
:103E400033E343E35FE30E94FB230E945F2360931D
:103E5000F7016C2FCC0F770B880B990B0E949723DF
:103E600023E333E343E35FE30E94FB230E945F23EA
:103E70006093F8011D1624F40E940D1D8093F90132
:103E80008091F90187FF05C00E940D1D81958093E7
:103E9000F901111624F40E940D1D8093FA018091FE
:103EA000FA0187FF05C00E940D1D81958093FA01DC
:103EB000DF91CF911F910C94331E9F3F09F08FCF5C
:103EC00097CFDF91CF911F910895E6EFF1E085E064
:103ED000DF011D928A95E9F71092F5011092F40125
:103EE000089587E296E00E9465051F9281E08F9316
:103EF0001F9285E08F9389ED95E09F938F930E94A9
:103F0000FE050F900F900F900F900F900F90089557
:103F10008330E9F128F4813061F0823009F10895AD
:103F2000853009F462C008F449C0863009F474C0D1
:103F3000089580911301262F30E0280F311D2F3F67
:103F4000310524F4680F6093130103C08FEF809351
:103F50001301809113011F928F9382E195E072C04B
:103F600080911201262F30E0280F311D2F3F31059F
:103F700024F4680F6093120103C08FEF8093120145
:103F8000809112011F928F9380E095E05BC0809139
:103F90001101262F30E0280F311D2F3F310524F469
:103FA000680F6093110103C08FEF8093110180911E
:103FB00011011F928F938DEE94E044C08091100107
:103FC000262F30E0280F311D2F3F310524F4680FD4
:103FD0006093100103C08FEF809310018091100156
:103FE0001F928F9388ED94E02DC080910F01262FB2
:103FF00030E0280F311D2F3F310524F4680F609306
:104000000F0103C08FEF80930F0180910F011F926A
:104010008F938FEB94E016C080910E01262F30E035
:10402000280F311D2F3F310524F4680F60930E01D6
:1040300003C08FEF80930E0180910E011F928F932A
:1040400084EA94E09F938F930E94FE050F900F9057
:104050000F900F900895833081F128F4813059F04A
:104060008230D1F00895853009F449C0B8F1863026
:1040700009F456C0089580911301681720F4861B37
:104080008093130102C010921301809113011F92BB
:104090008F9385E994E054C080911201681720F451
:1040A000861B8093120102C01092120180911201AE
:1040B0001F928F9383E894E043C0809111016817A9
:1040C00020F4861B8093110102C01092110180918F
:1040D00011011F928F9380E794E032C0809110010C
:1040E000681720F4861B8093100102C01092100103
:1040F000809110011F928F938BE594E021C08091F5
:104100000F01681720F4861B80930F0102C01092E4
:104110000F0180910F011F928F9382E494E010C0F1
:1041200080910E01681720F4861B80930E0102C057
:1041300010920E0180910E011F928F9387E294E0FE
:104140009F938F930E94FE050F900F900F900F90FA
:104150000895CF93C82F1F928F938CE297E09F937F
:104160008F930E94FE0581E090E0A0E0B0E0BC01EA
:10417000CD0104C0660F771F881F991FCA95D2F71B
:104180000E94BC180F900F900F900F90CF910C943D
:10419000AE14CF938732A8F58E3108F02BC1803151
:1041A00009F49FC0F8F4873009F464C0A8F486309D
:1041B00009F024C18091EC01817F8E7F8093EC0116
:1041C00081E397E00E9465058BE19AE00E94650516
:1041D00081E08093FC014CC08B30F1F18E3009F40A
:1041E0006CC00CC1863109F4B0C020F4813109F4EF
:1041F000EDC004C1893109F491C08B3109F449C083
:10420000FDC0883349F150F4893209F4F1C0853397
:1042100009F4EEC0873209F0F1C0EAC0833409F432
:10422000E7C028F48A3308F4E9C08953E4C088342D
:1042300009F0E4C00E94AE148AE09AE00E9465058D
:104240002FEF83ED90E3215080409040E1F700C0D4
:1042500000000E94661C0CC088E597E05CC081EFFE
:1042600099E00E9465058091EC0181608093EC01EA
:10427000C1E0C9C08091EC01C82FC17080FFEFCFB1
:104280008DEF99E00E9465058091EC01817F8E7F22
:104290003DC09091EC0191FBCC27C0F981E0C8278B
:1042A000892FC0FB81F98093EC01CC2319F084EEB7
:1042B00099E027C086ED99E02EC09091EC0192FB29
:1042C000CC27C0F981E0C827892FC0FB82F98093F1
:1042D000EC01CC2319F087EC99E013C087EB99E04F
:1042E0001AC09091EC0193FBCC27C0F981E0C8275C
:1042F000892FC0FB83F98093EC01CC2351F08BEA2A
:1043000099E00E9465058091EC0181608093EC0149
:104310007AC08EE999E00E946505AACF8FE899E0FE
:104320000E94650582E699E00E9465058BE299E0AE
:104330000E9465058EEF98E00E94650584EB98E089
:104340000E94650586E898E0E6CF88E798E00E943D
:1043500065050E94D00E1F928F938EE598E09F9383
:104360008F930E94FE0580910A011F928F9387E42C
:1043700098E09F938F930E94FE05809177011F9292
:104380008F9384E398E09F938F930E94FE05809122
:104390000B011F928F9381E298E09F938F930E946D
:1043A000FE050E94DF1B9F938F937F936F938AE09C
:1043B00098E09F938F930E94FE058DB79EB7469617
:1043C0000FB6F8949EBF0FBE8DBF52CF0E94AE14A1
:1043D000C0910B0181E0C827C0930B01CC2329F0C9
:1043E00080E098E00E9465050EC085EF97E093CFCE
:1043F00080E001C08D510E94A9203ACF83EF97E061
:104400000E946505C0E08C2FCF91089580E008954B
:1044100080E00895CF93C82F8091FC01813071F026
:1044200020F0823009F44BC042C1E0910C01F091C0
:104430000D018081823209F03CC107C0E0910C017E
:10444000F0910D018081823261F48C2F0E9406224E
:10445000811104C08C2F0E94C9202FC081E090E000
:104460002CC08C2F0E940822811126C0C431E1F09B
:1044700070F4CB3081F0C031D1F40E94711F84E21E
:1044800097E00E94650582E08093FC0115C0C93267
:1044900059F0C83361F481E397E00E94650588E232
:1044A00097E00E94650508C01092FC0104C182E2F9
:1044B00097E00E946505FFC081E08170FEC0C432B4
:1044C00028F5CE3108F0C1C0CB30A1F1D0F4C7300F
:1044D00009F0D3C08EE18093130182E3809312012F
:1044E0008AE08093110184E18093100188E0809339
:1044F0000F0188E280930E0188EC95E00E9465052B
:10450000BFC0C33149F1C431C1F0B7C0CB3409F4E5
:10451000A9C028F4C93289F0C83361F0AEC0C135F2
:1045200009F49EC0C23509F499C0CE3409F0A5C083
:104530006AE09EC00E94711FA3C08091FB01882386
:1045400019F01092FB019CC085ED95E00E94650575
:1045500081E08093FC01B1C08FEA95E00E9465057F
:104560008DE995E00E946505809113011F928F935C
:104570008AE995E09F938F930E94FE0588E995E074
:104580000E94650586E895E00E946505809112010C
:104590001F928F9383E895E09F938F930E94FE056F
:1045A00081E895E00E94650582E795E00E94650537
:1045B000809111011F928F938FE695E09F938F93C7
:1045C0000E94FE058DE695E00E9465058CE595E06C
:1045D0000E946505809110011F928F9389E595E0F7
:1045E0009F938F930E94FE0587E595E00E946505E5
:1045F00082E495E00E94650580910F011F928F93E0
:104600008FE395E09F938F930E94FE058DE395E0E5
:104610000E94650586E295E00E94650580910E0185
:104620001F928F9383E295E09F938F930E94FE05E4
:1046300081E295E00E9465058DB79EB748960FB65A
:10464000F8949EBF0FBE8DBF1BC0CE51EC2FF0E083
:10465000E25DFE4F80818093FB0112C061E003C0E8
:1046600061E006C06AE08091FB010E94881F08C0DB
:104670008091FB010E942B2003C086EC95E013C0C3
:104680008091FB01882369F01F928F9380EC95E065
:104690009F938F930E94FE050F900F900F900F90A5
:1046A00004C08DEB95E00E94650581E006C0109284
:1046B000FC0180E002C080E000CFCF9108950E940D
:1046C00066236894B1110C94F52308950E94DA23AF
:1046D00088F09F5798F0B92F9927B751B0F0E1F0C3
:1046E000660F771F881F991F1AF0BA95C9F714C073
:1046F000B13091F00E94F423B1E008950C94F423BA
:10470000672F782F8827B85F39F0B93FCCF38695AB
:1047100077956795B395D9F73EF490958095709508
:1047200061957F4F8F4F9F4F0895E89409C097FB85
:104730003EF490958095709561957F4F8F4F9F4F78
:104740009923A9F0F92F96E9BB279395F6958795BC
:1047500077956795B795F111F8CFFAF4BB0F11F47F
:1047600060FF1BC06F5F7F4F8F4F9F4F16C0882326
:1047700011F096E911C0772321F09EE8872F762F5C
:1047800005C0662371F096E8862F70E060E02AF09D
:104790009A95660F771F881FDAF7880F9695879589
:1047A00097F9089557FD9058440F551F59F05F3FF2
:1047B00071F04795880F97FB991F61F09F3F79F043
:1047C00087950895121613061406551FF2CF4695C5
:1047D000F1DF08C0161617061806991FF1CF869547
:1047E0007105610508940895E894BB27662777272B
:1047F000CB0197F908950E940E240C947F240E9407
:10480000712438F00E94782420F0952311F00C9444
:1048100068240C946E2411240C94F5230E94D22356
:1048200070F3959FC1F3950F50E0551F629FF00103
:10483000729FBB27F00DB11D639FAA27F00DB11D1C
:10484000AA1F649F6627B00DA11D661F829F2227A5
:10485000B00DA11D621F739FB00DA11D621F839F2C
:10486000A00D611D221F749F3327A00D611D231F02
:10487000849F600D211D822F762F6A2F11249F5750
:1048800050409AF0F1F088234AF0EE0FFF1FBB1F53
:10489000661F771F881F91505040A9F79E3F510512
:1048A00080F00C9468240C94F5235F3FE4F3983E69
:1048B000D4F3869577956795B795F795E7959F5FBC
:1048C000C1F7FE2B880F911D9695879597F908954E
:1048D00097F99F6780E870E060E008959FEF80ECB3
:1048E000089500240A941616170618060906089556
:1048F00000240A9412161306140605060895092EBC
:104900000394000C11F4882352F0BB0F40F4BF2B2A
:1049100011F460FF04C06F5F7F4F8F4F9F4F08956A
:10492000991B79E004C0991F961708F0961B881F01
:104930007A95C9F78095089597FB072E16F4009491
:1049400007D077FD09D00E94B62407FC05D03EF4BD
:10495000909581959F4F0895709561957F4F08952B
:10496000EE0FFF1F0590F491E02D0994AA1BBB1BCD
:1049700051E107C0AA1FBB1FA617B70710F0A61B5F
:10498000B70B881F991F5A95A9F780959095BC0180
:08499000CD010895F894FFCF5A
:104998000C07FD07DA07A60772070101CA012808F4
:1049A800140A321E404D362239F702AA0274025206
:1049B8000219028C01A501BE01D701F7010001020D
:0849C8000304050607080900BD
:106800000000000000000000040005000600070072
:10681000080009000A000B000C000D000E000F001C
:1068200010001100120013001400150016001700CC
:10683000180019001A001B001C001D001E001F007C
:10684000200021002200230024002500260027002C
:106850002800000035002B002C002D002E002F00FA
:1068600030002A00000033003400290036003700D1
:106870003800E00000000000000000000000000000
:106880000000000000000000000000000000000008
:1068900000000000000000000000000000000000F8
:1068A00000000000000000000000000000000000E8
:1068B00000000000000000000000000000000000D8
:1068C00000000000000000000000000000000000C8
:1068D00000000000000000000000000000000000B8
:1068E0000000000000000000310000000000000077
:1068F0000000E100E200E300F1A1E500E600E700AE
:106900000000000000000000EA4401000100E24431
:106910000100010001005500460054004A004B00F0
:10692000560057004700480001000100E9440100FB
:106930000100010001000100010001003A003B00DC
:106940003C003D003E003F0040004100420043004B
:10695000580000004C00390001004400450052007E
:1069600001000100000050004F0081404D004E002A
:1069700051000100000000000000000000000000C5
:106980000000000000000000000000000000000007
:1069900000000000000000000000000000000000F7
:1069A00000000000000000000000000000000000E7
:1069B00000000000000000000000000000000000D7
:1069C00000000000000000000000000000000000C7
:1069D00000000000000000000000000000000000B7
:1069E000000000000000000049000000000000005E
:1069F0000000010001000100010001000100010090
:00000001FF
